:020000040000FA
:06000000FE300C303A282E
:08000800A000030EA100831209
:10001000AA1503140B19031000308100A30DA40DC1
:10002000A50DA90B1C282A162508A8002408A7003E
:100030002308A6001930A9008B100B11210E830094
:06004000A00E200E0900D5
:0C007400203084008001840A80300402E7
:10008000031C3C281F30CE000130CA00CB0080305A
:10009000CD000E30F4003230D70083161F308505B6
:1000A000003086050B3087058312850186018701A4
:1000B000103083168E008312703083168F008312E7
:1000C0000030031799000313003003179A0003133D
:1000D0000C30970000309F00003083169F00831281
:1000E000183003179E000313003003179F000313FB
:1000F000803083168100831211309000043092000A
:100100007F308316920083120030950000308316F2
:100110009400831223309400A63083169800831233
:10012000003083169B00831210309800193083161C
:1001300099008312003083168C00831200308316DE
:100140008D00831200308B000D16CF2381018E01AC
:100150008F010B118B100B108C018D010D168B175D
:10016000E321B727311759219A22E920651AF02097
:10017000E51AEB202A1AF5208F080319B4288F01FD
:10018000E51A0717651A07150025B11B6821651ABE
:10019000F020E51AEB20A723982318227622651A6F
:1001A000F020E51AEB204F18A221651AF020E51A7D
:1001B000EB204F18B428AA19E328CC0BB428AA1AAC
:1001C000E7281930A900AA110C30CC00B42851211D
:1001D000B428640008006B080E0203180713080017
:1001E0006B080E020318071108002A12C1302802FA
:1001F000031D05292708BD002608BC0007303D0265
:100200000319CB277C23CF234C2928082706260255
:10021000031D0800F7302802031D11292708BF001D
:100220004C29A1302802031D18292708F0004C2969
:10023000A2302802031D1F292708C2004C29A7301D
:100240002802031D30292A10A71B2A1427087F39EA
:10025000EA002A1CEA012B142A1C2B10AB154C298E
:10026000C2302802031D4C292708C40064000D1E5B
:1002700037298B13440803178D0083168C130C1435
:1002800083120C080313C5008B177F3044022730FC
:100290000319C500CE164C29AA16AA110A30CC00A3
:1002A00008004F144F150B12831605118312051504
:1002B00008004F10CF101930A900AA12AA110A3055
:1002C000CC008316051583128B100B110B1608003A
:1002D000E61C080033080319080033083602031D22
:1002E000772934083702031D7729B1130800AF0AB4
:1002F00001302F02031D7F293308930008000730C7
:100300002F02031D86293408930008000D302F02A8
:10031000031D9029350803190800350893000800CB
:100320000E302F02031D08003308B6003408B70052
:10033000B301B401B501AF01B113311F0800C127EA
:10034000311308004F19AF29C9030F304905031DA8
:100350000800C9080319AF290515C90E08000511C1
:100360004F11CF1859294B184608CB1847084B197D
:1003700048084D05031DBF294430C900C22911306A
:10038000C900C2290310CD0C0318C729080080300A
:10039000CD000310CB0DCB19CE2908000130CB00C6
:1003A0001030CE1ACA00410840028030031DCA0036
:1003B0000310CA0D03184A144A084E050319CE2922
:1003C000E321CF140800C601C701C8014A1CEE2969
:1003D0007730C6004008C700C100142ACA1CF5299E
:1003E0006630C6004308C700142A4A1DFC29553050
:1003F000C6007108C700142ACA1D032A4430C6006B
:100400007508C700142A4A1E0A2A3330C600770826
:10041000C700142ACA1E08002130C6004408C700BD
:100420004508C800CE12080046084706C800080064
:10043000051CB80A0518B803380803194012031937
:10044000B80A3B083802031940160319B803851C83
:10045000B90A8518B90339080319C0110319B90A73
:100460003B0839020319C0150319B903851DBA0ADF
:100470008519BA033A08031940110319BA0A3B084F
:100480003A02031940150319BA038719C010871DD2
:10049000C0143F1886163F1C8612C219B823C21911
:1004A000552A2A1BB8232A1F0712E6195C2ABF1CEB
:1004B0008613BF188617602ABF1C8617BF188613BD
:1004C0003F1F6513401C672A3F1B672AE517710809
:1004D000C01800306619F100C318752A2B1C752A44
:1004E000053077024310031C43140800B11B0800B9
:1004F000E008031D08003108420601390319872A64
:10050000301342183017B127311042183114310816
:10051000420603390319932A3016B127B110C218C5
:10052000B114B2010800301E0800B20B08003012EE
:10053000B1270800EA080319A42AAB18AC2A6A08F4
:1005400095002A18A62A08009501080006162B1403
:10055000AB10421AAB1408002B1D08002B11D51844
:10056000F32AD70BB4283230D700D514AB19CB22DD
:100570008B131D3003178D0083168C130C148312FC
:100580000C080313DE006A0895002A1C0800AB1053
:10059000421AAB140800AB112130BF1C013E0317F7
:1005A0008D0083168C130C1483120C080313D800CF
:1005B0008B17203003178D0083168C130C148312B5
:1005C0000C080313DC008B1758085C07D9005C0784
:1005D000DA005C07DB006A087F3CDD000310DD0CFD
:1005E0000310DD0C0800DE08031DF82ADE030800F6
:1005F00058087702031C0A2B59087702031C0C2B9E
:100600005A087702031C0E2B5B087702031C102B81
:10061000D40A122BD00A122BD10A122BD20A122B77
:10062000D30A122B500851045204530454041039B5
:1006300003190800D601501AD614511A5615521A29
:10064000D615531A5616541AD616D001D101D20116
:10065000D301D401D5103230D7006A08ED005D0710
:100660005619ED005D07D619ED005D07561AED002D
:100670005D07D61AED006D08950008000030BD003A
:100680007108BC007C230800F10A720A7102031889
:10069000F1000800F103720AF11BF1070800640081
:1006A0000D1E502B8B13063003178D0083168C13F1
:1006B0000C1483120C0803138B173F1D3030F2000B
:1006C000F203701B792B700871020318712B031948
:1006D000712B71087002BF187202BF18013EF3003F
:1006E000080070087102BF1C7202BF1C013EF300BB
:1006F0000800FA30F30008000D123D0883120317BA
:100700008D00831203133C08831203178C00831699
:1007100003178C130C158B138B1B8B2B55308D00F3
:10072000AA308D008C148B170C1183120313080050
:10073000F40BA42B0E30F4009F147503F6009F18E1
:100740009F2B2A151E08F5008D309F0008009F146E
:100750009F18A82B2B158B1383161E0883128B173B
:10076000F7001E08C310031DC31411309F000800BA
:10077000AD132D13AD0B0800AC0A03302C02031C83
:10078000080007121E302E1C0A302C02031C080021
:10079000AE0A0130E61AAE000716AC01080064008C
:1007A0000D1ED02B8B13003003178D0083168C1376
:1007B0000C1483120C080313F1008B138B1BDD2B1D
:1007C000083003178D0083168C130C1483120C0849
:1007D0000313E6008B171C3003178D0083168C1350
:1007E0000C1483120C080313BB008B1708000708B6
:1007F000403A870008000708043A87000800070805
:10080000103A870008000608103A8600080006081B
:0E081000203A860008000608803A860008009C
:100A0000123060020318E00105308A006008820796
:100A10001A2D2E2DB82DD02DDC2DF52D1A2E2E2E83
:100A20005C2E962ED22EFD2E0D2F252F312F4A2FE4
:100A3000622F672F07170711FA01FB01EB01E5137E
:100A40004010C012651B08003F1F080065174F23A8
:100A5000F308031908000130E0000800AB1040144F
:100A6000B017B1272A17C31143138B13053003178F
:100A70008D0083168C130C1483120C080313EC00E6
:100A80008B178B13033003178D0083168C130C14F4
:100A900083120C080313F8008B178B130430031711
:100AA0008D0083168C130C1483120C080313F900A9
:100AB0008B178B130C3003178D0083168C130C14BB
:100AC00083120C080313FC008B178B130D300317D4
:100AD0008D0083168C130C1483120C080313FE0074
:100AE0008B178B130F3003178D0083168C130C1488
:100AF00083120C080313FD008B178B130E300317A2
:100B00008D0083168C130C1483120C080313FF0042
:100B10008B178B131B3003178D0083168C130C144B
:100B200083120C080313E4008B170130BF1C013E35
:100B30008B1303178D0083168C130C1483120C086F
:100B40000313EF008B171130BF1C013E8B130317EB
:100B50008D0083168C130C1483120C080313EE0003
:100B60008B176C08E100FF30EB000230E00008005A
:100B7000E516E10B08006C08E100EB0B0800E5123C
:100B80008B13133003178D0083168C130C148312F0
:100B90000C080313E1008B17E2010330E0000800AA
:100BA00007130711E20B0800E10B08006C08E100D5
:100BB000EB010430E00008006516E10B08006C084A
:100BC000E100EB0F0800EB0365128B1314300317E1
:100BD0008D0083168C130C1483120C080313E10090
:100BE0008B17E2010530E000080007130715E61C2B
:100BF000052EE1080319052EE61F3016E61B3017F7
:100C0000B127E20B0800E10B0800E61F3012E61BDB
:100C10003013B1278B13163003178D0083168C13F6
:100C20000C1483120C080313E1008B17E201063049
:100C3000E0000800E20B0800E10B08008B131830FD
:100C400003178D0083168C130C1483120C080313E6
:100C5000E1008B17E2010730E0000800C01606161D
:100C6000AB156E08EA00AB14661CAB10E514A027A8
:100C70002B14E20B0800E10B08000130E51BF30028
:100C8000AB1001307302031D4C2E6E08EA00AB144A
:100C9000661CAB10E5108F278B13193003178D00DE
:100CA00083168C130C1483120C080313E1008B17AA
:100CB000E2010830E0000800722778087502031886
:100CC000662E7F08FB02031C6B2E08007F08FB07C3
:100CD0000318852E0800FB010130E51BF300AB1063
:100CE00001307302031D7B2E6E08EA00AB14661CF4
:100CF000AB10E5108F27E20B0800E10B0800C315CD
:100D0000F3012A131130E0000800FB018B131A30A5
:100D100003178D0083168C130C1483120C08031315
:100D2000E1008B17E2010930E00008007227790822
:100D30007502031CA02E7F08FB02031CA52E0800D1
:100D40007F08FB070318AF2E0800FB01E20B080029
:100D5000E10B08004317F3011130E0000800BF1C4D
:100D60004423BF184A23F31BC22EF30BC22E6E0876
:100D7000EA00AB14661CAB10E5108F270A30E000C8
:100D8000FA0108008B13193003178D0083168C139A
:100D90000C1483120C080313E1008B17E2010830D6
:100DA000E00008002A1D08002A1175087602031CBD
:100DB000DE2E7C08FA02031CE52E08007E08BF1C0C
:100DC0007D08FA070318E72E0800FA010800FA0167
:100DD0008712EA012B10AB1089278B1317300317EA
:100DE0008D0083168C130C1483120C080313E1007E
:100DF0008B17E2010B30E00008003E23C012061200
:100E0000E20B0800B013B127E10B08006C08E10009
:100E1000FF30EB000C30E00008006516E10B080025
:100E20006C08E100EB0B080065128B1313300317FD
:100E30008D0083168C130C1483120C080313E1002D
:100E40008B17E2010D30E000080007130711E20BD9
:100E50000800E10B08006C08E100EB010E30E00037
:100E60000800E516E10B08006C08E100EB0F080034
:100E7000EB03E5128B13153003178D0083168C13CB
:100E80000C1483120C080313E1008B17E2010F30DE
:100E9000E000080007170711E61C5A2FE1080319A4
:100EA0005A2F661F3016661B3017B127E20B080059
:100EB000E10B0800661F3012661B3013B12710309B
:100EC000E00008002A1389270030E00008002A13F8
:100ED0008927B0138712EA012B10AB1006120030DD
:100EE000E0000800E51C0800E40B08008B131B3031
:100EF00003178D0083168C130C1483120C08031334
:100F0000E4008B17EA0A6F086A02031D0800E51067
:100F100008002430B3000030B400B11708002430BA
:100F2000B3008B131E3003178D0083168C130C1423
:100F300083120C080313B5008B17E527B1170800BF
:100F40002430B3008B131F3003178D0083168C13CE
:100F50000C1483120C080313B5008B17E527B11787
:100F600008000630B3003008B400B1170800143090
:100F7000AF00FE30B300D930B400FF30B500B11778
:100F800008001430AF00FE30B300E530B400FF308D
:100F9000B500B1170800B601FE30B300A130B400AF
:100FA000D327B1170800B5013C18B517BC18351781
:100FB0003C19B516BC1935163C1AB515BC1A3515B1
:100FC0003C1BB514BC1B35140800B4013518B4170C
:100FD000B51834173519B416B5193416351AB415B1
:0C0FE000B51A3415351BB414B501080017
:084000000B00000002000700A4
:02400E00CC03E1
:1042000000007E007E00AA0096000A001800FF0051
:104210008700FF00FF00FF0041002E0014002E0069
:1042200000003200320002001400150016003700B2
:104230000600190080005A00FF0000000100600025
:10424000050040004000FF00FF00FF00FF00FF00EE
:10425000FF00FF00FF00FF00FF00FF00FF00FF0066
:10426000FF00FF00FF00FF00FF00FF00FF00FF0056
:10427000FF00FF00FF00FF00FF00FF00FF00FF0046
:10428000FF00FF00FF00FF00FF00FF00FF00FF0036
:10429000FF00FF00FF00FF00FF00FF00FF00FF0026
:1042A000FF00FF00FF00FF00FF00FF00FF00FF0016
:1042B000FF00FF00FF00FF00FF00FF00FF00FF0006
:1042C000FF00FF00FF00FF00FF00FF00FF00FF00F6
:1042D000FF00FF00FF00FF00FF00FF00FF00FF00E6
:1042E000FF00FF00FF00FF00FF00FF00FF00FF00D6
:1042F000FF00FF00FF00FF00FF00FF00000027009D
:00000001FF
